BL51 BANKED LINKER/LOCATER V6.22                                                        09/28/2022  19:54:06  PAGE 1


BL51 BANKED LINKER/LOCATER V6.22, INVOKED BY:
C:\KEIL_V4\C51\BIN\BL51.EXE .\Release\system_FE81001.obj, .\Release\STARTUP.obj, .\Release\main.obj TO .\Release\Sample_
>> DrvWDT REGFILE (.\Release\Sample_DrvWDT.ORC) PRINT (.\Sample_DrvWDT.m51) RAMSIZE (256) CODE (0X0000-0X1FFF) XDATA (0X
>> 8000-0X83FF)


MEMORY MODEL: SMALL


INPUT MODULES INCLUDED:
  .\Release\system_FE81001.obj (SYSTEM_FE81001)
  .\Release\STARTUP.obj (?C_STARTUP)
  .\Release\main.obj (MAIN)
  C:\KEIL_V4\C51\LIB\C51S.LIB (?C_INIT)
  C:\KEIL_V4\C51\LIB\C51S.LIB (?C_IBP)


LINK MAP OF MODULE:  .\Release\Sample_DrvWDT (SYSTEM_FE81001)


            TYPE    BASE      LENGTH    RELOCATION   SEGMENT NAME
            -----------------------------------------------------

            * * * * * * *   D A T A   M E M O R Y   * * * * * * *
            REG     0000H     0008H     ABSOLUTE     "REG BANK 0"
            DATA    0008H     0006H     UNIT         ?DT?_DELAY?MAIN
            DATA    000EH     0001H     UNIT         ?DT?WDTISR?MAIN
            DATA    000FH     0001H     UNIT         ?DT?MAIN
            DATA    0010H     0001H     UNIT         ?C?LIB_DATA
            IDATA   0011H     0001H     UNIT         ?STACK

            * * * * * * *   C O D E   M E M O R Y   * * * * * * *
            CODE    0000H     0003H     ABSOLUTE     
            CODE    0003H     0036H     UNIT         ?PR?WDTCLKINIT?MAIN
            CODE    0039H     0001H     UNIT         ?PR?SYSTEMINIT?SYSTEM_FE81001
                    003AH     0001H                  *** GAP ***
            CODE    003BH     0003H     ABSOLUTE     
            CODE    003EH     009DH     UNIT         ?C_C51STARTUP
            CODE    00DBH     008BH     UNIT         ?PR?MAIN?MAIN
            CODE    0166H     0054H     UNIT         ?PR?WDTINIT?MAIN
            CODE    01BAH     003BH     UNIT         ?PR?_DELAY?MAIN
            CODE    01F5H     002BH     UNIT         ?PR?WDTISR?MAIN
            CODE    0220H     0004H     UNIT         ?C_INITSEG



OVERLAY MAP OF MODULE:   .\Release\Sample_DrvWDT (SYSTEM_FE81001)


SEGMENT
  +--> CALLED SEGMENT
---------------------
?C_C51STARTUP
  +--> ?PR?MAIN?MAIN
  +--> ?C_INITSEG

?PR?MAIN?MAIN
  +--> ?PR?_DELAY?MAIN
BL51 BANKED LINKER/LOCATER V6.22                                                      09/28/2022  19:54:06  PAGE 2


  +--> ?PR?WDTCLKINIT?MAIN
  +--> ?PR?WDTINIT?MAIN



SYMBOL TABLE OF MODULE:  .\Release\Sample_DrvWDT (SYSTEM_FE81001)

  VALUE           TYPE          NAME
  ----------------------------------

  -------         MODULE        SYSTEM_FE81001
  C:0000H         SYMBOL        _ICE_DUMMY_
  C:0039H         PUBLIC        SystemInit
  -------         PROC          SYSTEMINIT
  C:0039H         LINE#         38
  C:0039H         LINE#         39
  C:0039H         LINE#         41
  -------         ENDPROC       SYSTEMINIT
  -------         ENDMOD        SYSTEM_FE81001

  -------         MODULE        ?C_STARTUP
  C:003EH         SEGMENT       ?C_C51STARTUP
  I:0011H         SEGMENT       ?STACK
  C:0000H         PUBLIC        ?C_STARTUP
  D:00E0H         SYMBOL        ACC
  D:00F0H         SYMBOL        B
  D:0083H         SYMBOL        DPH
  D:0082H         SYMBOL        DPL
  N:0001H         SYMBOL        IBPSTACK
  N:0100H         SYMBOL        IBPSTACKTOP
  N:0080H         SYMBOL        IDATALEN
  C:0041H         SYMBOL        IDATALOOP
  N:0000H         SYMBOL        PBPSTACK
  N:0100H         SYMBOL        PBPSTACKTOP
  N:0000H         SYMBOL        PDATALEN
  N:0000H         SYMBOL        PDATASTART
  N:0000H         SYMBOL        PPAGE
  N:0000H         SYMBOL        PPAGEENABLE
  D:00A0H         SYMBOL        PPAGE_SFR
  D:0081H         SYMBOL        SP
  C:003EH         SYMBOL        STARTUP1
  N:0000H         SYMBOL        XBPSTACK
  N:0000H         SYMBOL        XBPSTACKTOP
  N:0800H         SYMBOL        XDATALEN
  C:004CH         SYMBOL        XDATALOOP
  N:8000H         SYMBOL        XDATASTART
  C:0000H         LINE#         126
  C:003EH         LINE#         133
  C:0040H         LINE#         134
  C:0041H         LINE#         135
  C:0042H         LINE#         136
  C:0044H         LINE#         140
  C:0047H         LINE#         141
  C:0049H         LINE#         145
  C:004BH         LINE#         147
  C:004CH         LINE#         148
  C:004DH         LINE#         149
BL51 BANKED LINKER/LOCATER V6.22                                                      09/28/2022  19:54:06  PAGE 3


  C:004EH         LINE#         150
  C:0050H         LINE#         151
  C:0052H         LINE#         170
  C:0055H         LINE#         185
  C:0058H         LINE#         196
  -------         ENDMOD        ?C_STARTUP

  -------         MODULE        MAIN
  C:0000H         SYMBOL        _ICE_DUMMY_
  D:0090H         PUBLIC        P1
  D:00B0H         PUBLIC        P3
  C:0166H         PUBLIC        WDTInit
  D:00A8H         PUBLIC        IE
  C:01BAH         PUBLIC        _delay
  D:00B8H         PUBLIC        IP
  C:0003H         PUBLIC        WDTClkInit
  C:00DBH         PUBLIC        main
  D:0098H         PUBLIC        SCON
  D:0088H         PUBLIC        TCON
  D:000FH         PUBLIC        cnt
  C:01F5H         PUBLIC        WDTISR
  D:00C8H         PUBLIC        T2CON
  D:00D0H         PUBLIC        PSW
  -------         PROC          _DELAY
  D:0008H         SYMBOL        cnt
  -------         DO            
  D:000AH         SYMBOL        i
  D:000CH         SYMBOL        j
  -------         ENDDO         
  C:01BAH         LINE#         38
  C:01BEH         LINE#         39
  C:01BEH         LINE#         42
  C:01CFH         LINE#         43
  C:01F4H         LINE#         45
  -------         ENDPROC       _DELAY
  -------         PROC          WDTISR
  -------         DO            
  D:000EH         SYMBOL        int_stat
  -------         ENDDO         
  C:01F5H         LINE#         57
  C:0202H         LINE#         60
  C:0209H         LINE#         61
  C:020FH         LINE#         67
  C:0215H         LINE#         68
  -------         ENDPROC       WDTISR
  -------         PROC          WDTINIT
  C:0166H         LINE#         80
  C:0166H         LINE#         81
  C:0166H         LINE#         83
  C:016CH         LINE#         86
  C:0182H         LINE#         89
  C:0198H         LINE#         92
  C:01A3H         LINE#         93
  C:01AEH         LINE#         94
  C:01B9H         LINE#         95
  -------         ENDPROC       WDTINIT
  -------         PROC          WDTCLKINIT
BL51 BANKED LINKER/LOCATER V6.22                                                      09/28/2022  19:54:06  PAGE 4


  C:0003H         LINE#         107
  C:0003H         LINE#         108
  C:0003H         LINE#         110
  C:000EH         LINE#         113
  C:0024H         LINE#         116
  C:002DH         LINE#         119
  C:0038H         LINE#         120
  -------         ENDPROC       WDTCLKINIT
  -------         PROC          MAIN
  C:00DBH         LINE#         132
  C:00DBH         LINE#         133
  C:00DBH         LINE#         135
  C:00E6H         LINE#         138
  C:0107H         LINE#         141
  C:0128H         LINE#         144
  C:012DH         LINE#         145
  C:0132H         LINE#         146
  C:0137H         LINE#         147
  C:013EH         LINE#         149
  C:0144H         LINE#         150
  C:014AH         LINE#         151
  C:0150H         LINE#         152
  C:0157H         LINE#         155
  C:015AH         LINE#         158
  C:015DH         LINE#         161
  C:0163H         LINE#         163
  C:0163H         LINE#         164
  C:0163H         LINE#         166
  C:0165H         LINE#         167
  -------         ENDPROC       MAIN
  -------         ENDMOD        MAIN

  -------         MODULE        ?C_IBP
  D:0010H         PUBLIC        ?C_IBP
  -------         ENDMOD        ?C_IBP



FUNCTION REGISTER MASKS


FUNCTION . . . . . REG MASK
---------------------------

MAIN . . . . . . . @0xf303
SYSTEMINIT . . . . @0x8000
WDTCLKINIT . . . . @0xe301
WDTINIT. . . . . . @0xe301
WDTISR . . . . . . @0xa301
_DELAY . . . . . . @0xf000

*** WARNING L16: UNCALLED SEGMENT, IGNORED FOR OVERLAY PROCESS
    SEGMENT: ?PR?SYSTEMINIT?SYSTEM_FE81001

Program Size: data=18.0 xdata=0 code=547
LINK/LOCATE RUN COMPLETE.  1 WARNING(S),  0 ERROR(S)
